:060000008A110A122F28EC
:100008008C00030EB700B70E0A08B8000408B90040
:10001800BF018A110A120B1D28283D0883120313F9
:100028008100C330BD004E30BE070318BD0ABD09AC
:10003800BD0A3F14C00A0319C10A0B11FF30C81BBF
:100048002828C707031CC8070D08BA000E08BB00FC
:100058000F08BC00882A8B138312031385018601BD
:10006800FF308316850086009A0187308100C330EF
:10007800BD00BE0183128100A0308B00C201FF3099
:10008800C501C601C700C8002B2A1408003A031D81
:100098005028050897005228060897001308003AC8
:1000A800031D592817089B0061281308013A031DEE
:1000B80061281708FF3A9B00612812290130970030
:1000C8001808170598000030F83E031C6D289801A1
:1000D80075280739031975280310980CFF3E031D6E
:1000E800702818089B00782815291B089100130808
:1000F800003A031D82281B08970085281B08FF3A31
:1001080097001408003A031D8D28170883128600EB
:1001180090281708831285001D088A001C08820091
:100128001B0892001308003A031D9D281B0897001E
:10013800A0281B08FF3A97001408003A031DA828B6
:10014800170883128500AB281708831286001D083C
:100158008A001C088200013097002308F83E031C1F
:10016800B7289701BF2807390319BF280310970D2F
:10017800FF3E031DBA28220898002308F83E031CF6
:10018800C7289801CF2807390319CF280310980DDD
:10019800FF3E031DCA281708A600A60926089105D0
:1001A8001808910411089B0000309D00DD309C0068
:1001B800792825088A002408820001309700013038
:1001C800F83E031CE9289701F12807390319F1289B
:1001D8000310970DFF3E031DEC282208980003101A
:1001E800980D1708A500A509250892051808920476
:1001F80012089B0001309D0003309C0094282408BD
:100208008A00230882000030940001309300FF30F8
:1002180083168500860191012C2A49281B0898001D
:1002280062281B0897001708A2001A294B292208E0
:100238002304240425040314031D031003183B2975
:10024800FF30A2078E018F018E0DFF30A3078F0D9F
:10025800FF30A4070318A50AFF30A5070E08A30757
:1002680003188F0A0F08A4070318A50A1B292708D3
:100278008A002608820096010130A2000130A400FD
:100288004730A300E128FE3099009903112922087C
:1002980098001808013A031D60291608FF3A031D43
:1002A8005E29A2010130A4005B30A300E1281608F2
:1002B800AC008629960A7429A2010130A400663090
:1002C800A300E128A501A4010330A300E830A2009F
:1002D8000130A7007130A6001B291608AC0086293A
:1002E8001908003A031D7B291608AC008629A501C8
:1002F800A401A3010830A2000130A7008530A600A0
:100308001B294929622A3108AC000130A2000230B9
:10031800A3000130A5009230A400AF28A20100304C
:10032800A3000130A5009A30A400AF28A501A401BC
:100338002730A3001030A2000130A700A530A60086
:100348001B290130A2000130A3000130A500AE3006
:10035800A400AF28A501A4010B30A300B830A20067
:100368000130A700B930A6001B29A2010130A30063
:100378000130A500C130A400AF28A501A401273091
:10038800A3001030A2000130A700CC30A6001B2922
:10039800A2010230A3000130A500D430A400AF2888
:1003A800033096001608003C0318292A96032C08E7
:1003B800803997002C089700970D9701970D17081B
:1003C800A2000030A3000130A500EC30A400AF2843
:1003D800A501A4012730A3001030A2000130A70016
:1003E800F730A6001B290130A2000130A30002301B
:1003F800A5000030A400AF28A501A4010B30A3007C
:10040800B830A2000230A7000B30A6001B29A201B9
:100418000130A3000230A5001330A400AF28A501C5
:10042800A4012730A3001030A2000230A7001E301C
:10043800A6001B29A2010030A3000230A500263027
:10044800A400AF280310AC0DD6292A2A792A072937
:1004580001308500B201013032020318352AB20A90
:10046800522AB2010130A2000330A3000230A500D5
:100478003F30A400AF28A501A401C330A300503029
:10048800A2000230A7004A30A6001B29A2010330AF
:10049800A3000230A5005230A400AF283208B100F2
:1004A8000310B10D0310B10D1C30B10631089B00CB
:1004B80002309D0061309C0094283F292C08B1002F
:1004C800E030B10531089B0002309D006D309C0082
:1004D8007928A501A401C330A3005030A20002303E
:1004E800A7007830A6001B298729A501A40103309D
:1004F800A300E830A2000230A7008430A6001B2920
:100508002F2A8A110A1200283C088F003B088E0007
:100518003A088D003908840038088A0037088300B3
:060528008C0E0C0E090010
:02400E000300AD
:00000001FF
